:020000040000FA
:040000000D2019288E
:080008008C00030E8D00322074
:100010000D0E83008C0E0C0E0900830183169730A1
:100020008100E0308500860183128501860181010F
:10003000080000308600003085001E288E018F01E8
:100040009001900A81018B018B168B1701083F39B3
:1000500091000E0811020301031CFF3086000F39C6
:10006000850026280B1D08000B1180308F07031D0B
:10007000080010088E07901B452841300E02031C13
:1000800008008E03FF30900008008E1F08008E0AC3
:06009000013090000800A1
:084000000000000000000100B7
:02400E00FA3F77
:00000001FF
